:020000040000FA
:100000002E288207003400340034003400341B34BE
:1000100077344034003435346734E03400346A34A3
:10002000CF34C03400349A341D3420340034D534F5
:100030009F34803401341334B234203401344034DA
:100040006F34403401347B34CA3490340134AB34DF
:100050003F3400340134C934C33480348B018316F7
:100060008113FB308500860183120511B520F8202D
:10007000051A3B28EE2189018D230808A3008D2352
:100080000808A4008D230808A5008D230808A600F1
:100090008D2308088C008D2308088D008D23080807
:1000A0008E008D2308088F00E52213238922C022A9
:1000B000CB22CB220508B30003303305B200B001D8
:1000C0004030AF00B401B6018B21B31969288A20F2
:1000D00064289D019C019B0101309A00331A7A2803
:1000E000E8309A0003309B007A2803109A0D9B0D8C
:1000F0009C0D9D0DAF0DB00D031C7528B418822802
:10010000782184283B215321E52213238922C02210
:10011000CB226428B41896280430B602EB30360798
:10012000031C94281430B600A3209D280430B60781
:10013000EB3036070318B601A320E52213238922EA
:10014000C022CB220800360801208F00B60A3608EC
:1001500001208E00B60A360801208D00B60A360846
:1001600001208C000330B60208009D230330860076
:1001700006169D230612033086000616A0230612DB
:10018000033086000616A0230612023086000616EB
:10019000A323061228305E2308305E2301305E233D
:1001A00006305E230C305E230800C0305E23203012
:1001B00062232030622320306223203062232030EB
:1001C00062232030622320306223203062232030DB
:1001D00062232030622320306223203062232030CB
:1001E0006223203062232030622320306223080003
:1001F00081305E2356306223463062234F306223C3
:10020000203062234430622344306223533062231F
:10021000203062234130622344306223393062232C
:100220003830622335306223313062239223C0306C
:100230005E234630622352306223453062235130C0
:10024000622355306223453062234E3062234330AF
:1002500062234530622320306223523062235830BB
:1002600062232030622353306223443062235230B1
:100270006223922308001A088C07031C44298D0F5F
:1002800044298E0F44298F0A1B088D07031C4B2914
:100290008E0F4B298F0A1C088E07031C50298F0ACA
:1002A0001D088F070800FF300F0703186F29003063
:1002B0000F02031C77291B300E0703186F29E43047
:1002C0000E02031C77291E300D0703186F29E13039
:1002D0000D02031C7729C0300C02031C7729C030A3
:1002E0008C00E1308D00E4308E0000308F0008007B
:1002F0009A099B099C099D099A0F83299B0F8329C1
:100300009C0F83299D0A3B218F1F8A298C018D0117
:100310008E018F010800B0014030AF00B421B01B46
:1003200095290830AF070318B00A0508B300033059
:100330003305B100320603198E290310B20D3108BE
:10034000B20632080239B50034060319AC29350863
:10035000B4003108B2008E29B401B21CB1290230B8
:10036000B4003108B2000800051EB9298519C22958
:10037000BE298519C0293818C429D7293814ED2970
:100380003810ED29B801ED291030B900051ACD2932
:100390009A23B90BC6297A22ED299D010F309C00C2
:1003A00042309B0040309A003B215321E829103015
:1003B000B9008519E0299A23B90BD9297A22ED29A8
:1003C0009D010F309C0042309B0040309A00782104
:1003D000E52213238922C022CB22080080308C0022
:1003E00096308D0098308E0000308F0089018D236B
:1003F0000808A3008D230808A4008D230808A50081
:100400008D230808A600E5221323D520C030AB00B9
:100410005E232030AB0062234330AB0062234130C7
:10042000AB0062234C30AB0062234930AB00622347
:100430004230AB0062235230AB0062234130AB004C
:1004400062235430AB0062234930AB0062234F304B
:10045000AB0062234E30AB0062232E30AB00622330
:100460002E30AB0062232E30AB0062232030AB0075
:1004700062238922CB228B219D019C019B0110309C
:100480009A003319452A80309A000000B418532A84
:100490009A099B099C099D099A0F532A9B0F532A7D
:1004A0009C0F532A9D0A1A08A307031C5C2AA40F59
:1004B0005C2AA50F5C2AA60A1B08A407031C632A52
:1004C000A50F632AA60A1C08A507031C682AA60A0A
:1004D0001D08A607051E392A8901230888008023E4
:1004E00024088800802325088800802326088800A7
:1004F00080230800043089000C08880080230D0840
:10050000880080230E08880080230F08880080233D
:100510000800950196019701980199012030A000EB
:100520002308A7002408A8002508A9002608AA0077
:100530000310271CB22A0C089607031CA42A970F45
:10054000A42A980FA42A990A0D089707031CAB2A1E
:10055000980FAB2A990A0E089807031CB02A990A2B
:100560000F089907990C980C970C960C950CAA0CEF
:10057000A90CA80CA70CA00B982A01309900080020
:100580000310950D960D970D980D0310950D960D72
:10059000970D980D0800153084000008A20008305F
:1005A000A100A20C031CD82A861506150611DB2A09
:1005B000861106150611A10BD12A840A1A300402ED
:1005C000031CCD2A86178613080020309E00900158
:1005D000910192019301940103108C0D8D0D8E0DEC
:1005E0008F0D03180C14900D910D920D930D940D19
:1005F0009E03031DFC2A0800103084000823840A8F
:100600000823840A0823840A0823840A0823EC2A7E
:10061000033000079F009F198000303000079F00C3
:100620009F1B8000080080305E2320306223130E61
:100630000F39303E622313080F39303E62232C30CD
:100640006223120E0F39303E622312080F39303EFA
:100650006223110E0F39303E62232E3062231108BF
:100660000F39303E6223100E0F39303E62231008DE
:100670000F39303E6223203062234D3062234830F0
:1006800062237A30622320306223080086018316B9
:1006900008308600831206138616FF30AD0006165A
:1006A0000608AC0006120000000006160000061244
:1006B000AD0303195D2BAC194F2B0800AB00B7013C
:1006C0000613652BAB0037140617462386018316E5
:1006D0000030860083128612061337180617F03092
:1006E00086052B0E0F398604061600000612F03020
:1006F00086052B080F39860406160000061208002E
:100700008316081555308900AA3089008814881886
:10071000872B08118312890A080083160814831294
:10072000890A0800972397239723972308009A2381
:100730009A230800FF30AD00A82B8030AD00A82B15
:100740004030AD00A82B2030AD00A82B1030AD00FC
:0E075000FF30AE00AE0BAA2BAD0BA82B08009D
:084000007F007F007F007F00BC
:02400E00F13F80
:10420000DE006500DC001700C000CF006A0000007F
:10421000000000000000000000000000000000009E
:10422000000000000000000000000000000000008E
:10423000000000000000000000000000000000007E
:10424000000000000000000000000000000000006E
:10425000000000000000000000000000000000005E
:10426000000000000000000000000000000000004E
:10427000000000000000000000000000000000003E
:00000001FF
